:02000000C22814
:10000800A00003088301B7000408B8000A08B90073
:100018008A015408C1005E08C2005F08C300550881
:10002800C6005608C5005708C4005808C700590834
:10003800C8005A08C9005B08C0005C08BF005D081A
:10004800BE003C08BA003D08BB0083128B1C9D28EB
:10005800012336225408AD005508AE005608AF00FB
:10006800A108031D3E282D08A2002E08A3002F0872
:10007800A4008E28210B8E282208D7002308D80038
:100088002408D9002D08D4002E08D5002F08D60042
:1000980072215408B0005508B1005608B200300863
:1000A800D4003108D5003208D6002E235408D700D2
:1000B8005508D8005608D9002508D4002608D500C8
:1000C8002708D600A32103188528D701D801D9010C
:1000D8003008D4003108D5003208D600A32103180F
:1000E8007F282508D7002608D8002708D9002230FD
:1000F80084004F218E282508D7002608D800270815
:100108008A283008D7003108D8003208D9002230B0
:100118008400512183122208D4002308D500240822
:10012800D600FA215408B3005508B400A7228B1052
:1001380083124108D4004208DE004308DF00460865
:10014800D5004508D6004408D7004708D800480815
:10015800D9004908DA004008DB003F08DC003E0807
:10016800DD003A08BC003B08BD00380884003908A7
:100178008A0037088300A00E200E09002130840071
:100188003730CE208316FF2390008301762A040699
:100198008001840A0406031DCB28640000348312FE
:1001A800BC00BD1BDE283D088A003C08BC0A0319B8
:1001B800BD0A820083133D1883173C08BC0A8400DB
:1001C800000808000310FF30D407D409031CD50722
:1001D800D509031CD607D609031CD707D709080079
:1001E800D501D601D701D41F222AD503D603D703B8
:1001F8001D2AD501D601D701222ADC01550D560D3D
:10020800DA005A0803190C29DC0DD601D5170800A5
:10021800D401D501D6010034DC10580D590DDB008E
:100228005B0803191C290318DC14D901D817080026
:10023800DB01D701D801D90108005A0803190C2994
:10024800D513DC0C5A0CD6000318D517392ADA084E
:10025800031D3F29D401D501D601392A56030319B4
:10026800D40A0319D50A0319D60A0310D60CD50CDB
:10027800D40CDA0A2B29D608031D32295408550450
:1002880003192E29D51B2129DA0303192E29031056
:10029800D40DD50D46298030D9060008D400840A2B
:1002A8000008D500840A0008D60075295A085B02A0
:1002B800031C6929031908000310D60CD50CD40CAB
:1002C800DA0A5A085B025E290310D90CD80CD70C3D
:1002D800DB0A5A085B060319080068298030D9062A
:1002E8008401012110215A215C1C8229D409D509D5
:1002F800D609D40A0319D50A0319D60ADC1C8C2995
:10030800D709D809D909D70A0319D80A0319D90A64
:100318005708D40758080318580FD5075908031861
:10032800590FD607DC01D61F2B29D409D509D609C0
:10033800D40A0319D50A0319D60A5C142B295608BE
:10034800590680390319AC29590D59080138080094
:10035800D61359087F395602031DBA295808550281
:10036800031DBA2957085402031908000308023864
:10037800D91B013A83000318803808008401012141
:100388001021DD01DE01DF01DA08031908005B082E
:10039800031908005A02773EDA005C0CDC061830B4
:1003A800D9000310DD0DDE0DDF0D5608031DE4290D
:1003B80058085502031DE22957085402031CEE2968
:1003C8005708D4025808031C580FD502031CD6033B
:1003D8005D140310D40DD50DD60DD90BD5295D08A4
:1003E800D4005E08D5005F08D6002B2984010121BE
:1003F800D7018230DA07DA1B0C29F030DA07DA1B6A
:10040800162A18305A0203180C29DA08031D0F2A75
:100418005C18E6200800DA030310D40DD50DD60DBC
:10042800D70D092A0310D60CD50CD40CDA0F162ACE
:100438000C2AD71F222A5C14E620232ADC018E30DE
:10044800DA008401D70803192B290310D70CD60C1E
:10045800D50CD40CDA0A262AD601D51BD6035608A1
:10046800D7001D2AD601D701222A8408031900348F
:1004780056088000840355088000840354088000CF
:1004880000348312A8002808A9002908AA008316A6
:100498009C184B2A8312280383169B00702A831604
:1004A8009C18532A83122A08BD002908D3208316D2
:1004B8009A008312A90A0319AA0A83169B0A031031
:1004C8008B1B03148B131C1555309D00AA309D00FF
:1004D8009C141C1103188B178312AA032A0F532A82
:1004E800280808008312A80183121A230030A900E3
:1004F8000330AA005730CB22D401A030D5004130B8
:10050800D600C2215408A5005508A6005608A70021
:10051800A101831601170B160B118B108B17982A44
:100528000B1D982AA80A0B1183122808D400FD2055
:10053800D7011630D8004230D900A321031C942AD1
:10054800A101A10AA62A023083123402BC30031981
:100558003302031C080008303402FD30031933024B
:10056800031808003408D5003308D400D409D50985
:100578005408B5005508B6008F0035088E000C10D9
:10058800101485140C1CC62A85101010080083123C
:10059800AB00AC00290883169B009C1CE02AD12ADA
:1005A80083161C1483122C08840083161A088000F2
:1005B8008312AC0A83169B0A8312AA032A0FD42A31
:1005C8002B0808008C3083129F00183083169F0078
:1005D80083121F142130AA00AA0BF02A9F149F1817
:1005E800F32A1E08A90083161E088312A8001F10EC
:1005F8002908D5002808D400080083128F018E012D
:1006080010140519052B10100F088312B400B3013C
:100618000E08D400D5013308D4070318D50A3408C6
:10062800D5072730D4070318D50A08008316FF23F7
:10063800900083123D308316850018309F00FF30EC
:100648008312990004309000473083168100951476
:0806580083120800D6130034E0
:084000000000080001000000AF
:02400E00843FED
:0642000000002000410057
:00000001FF
